:030000000203E216
:030003000203CE27
:03000B00020228C6
:10010000758921759852758780758DFED28E223043
:1001100099FDC299F599227F057E00209807DEFBA4
:10012000DFF774FF22C298E599223098FDC298E566
:100130009912010F2212013F90063D1205E122742F
:100140000D12010F740A12010F22741312010F22F3
:10015000741112010F22742012010F22C3FE944168
:100160005005EEC3943022C3EE943722EDC42C2206
:1001700012012A12015CFD12012A12015CFC12011B
:100180006C22540FFAC3940A5004EA243022EA2461
:100190003722F5F0120182FCE5F0C4120182FD2243
:1001A000120192ED12010FEC12010F2208E6C45465
:1001B000F0F918E6C4FA540F2908F6EA54F018F6D4
:1001C00022C3E53D253DF53DE53E353EF53E227534
:1001D000360075370075380079007F101201C15064
:1001E000119001F8C378367E03E99336D4F6A3085C
:1001F000DEF7090909DFE52268270384630192819C
:10020000009640004820002410001205005602000D
:1002100028010064000032000016000008000004FD
:100220000000020000010000C0D0C0E0C0F0C082A9
:10023000C08375D008758C8B852F8A1202FD052529
:10024000E525B40A21052CE52CB40507752C00D250
:100250001AC2B7120367301803120326752500E58A
:10026000262401D4F526E526B460103019031203C4
:1002700026752600E5272401D4F527E527B4600A72
:10028000752700E5282401D4F528E528B4240A754B
:100290002800E5292401D4F52912038CE529B5F0BD
:1002A0000A752901E52A2401D4F52AE52AB4130A9E
:1002B000752A01E52B2401D4F52BD083D082D0F010
:1002C000D0E0D0D0321201561201567E0190074381
:1002D0001205E178217F08E6F4F590F4F5F0E5F0F9
:1002E00033F5F0400A742D12010F12015680087484
:1002F0004F12010F120156DFE508DED922301A0F26
:10030000E52D04F52DB40107752D00D2B7C21A22D0
:100310007F00C2A27E50DEFED2A27E50DEFEDFF261
:1003200022540F24302212013FE5291201A0742D1E
:1003300012010FE52A1201A0742D12010F7425126B
:1003400001A0E52B1201A0120156E5281201A074AC
:100350003A12010FE5271201A0743A12010FE526A7
:100360001201A01202C5227830E6B40F012220B596
:1003700003B5291208E6B5280E08E6B5270A08E6EF
:10038000F521F4F590220808080880DDE52AC394D9
:10039000104007E52AC394068002E52A149003A6BC
:1003A00093F5F005F02231283130313031313031E0
:1003B00030317F067830E6120321F608DFF8227F1D
:1003C000067835E612010F18DFF912013F22C0E06E
:1003D000D20FE521F4F590D0E032C3E6970809E6A4
:1003E0009722758160752D007590FFC218C21A752D
:1003F0002500752C00752F92E52EB42502801B7503
:100400002E2575300F752600752730752812752931
:1004100029752A04752B37752100D2AFD2A9D2A82D
:10042000758901120100D2B99005F51205E1758CAC
:100430008B758A92D28C3098FDC298E599B4410EA2
:1004400012012AB4540812012AB40DFA80E844209B
:10045000B46F028047B474028049B47A028048B411
:100460006502805EB464028077B43F030204FEB488
:10047000730302050AB4700302050FB47203020588
:1004800072B463030205C9B42F030205D812013503
:10049000020436758A92758C8BD28C22C218120196
:1004A000358093D218808F12013FE52F1201A012E0
:1004B000013F743F12010F120170F52F1201350236
:1004C00004369007521205E1120170F528120170EE
:1004D000F527120170F526120326120135020436A3
:1004E00090076A1205E1120170F529120170F52AD0
:1004F000120170F52B120326120135020436900604
:10050000401205E1120135020436B219020436C266
:100510008C9007281205E112013F783012012AB4AD
:100520003AFA120170B40002803212012A120170EC
:10053000F612012A08120170F608120170F6087FFF
:100540000812012A12012AB43003C38001D3E63312
:10055000F6DFEE12012AB40AFA0880C0760F120103
:100560002AB40AF89007171205E1120135D28C025D
:10057000043612013F7830E6B40F08900782120566
:10058000E180401201A012015608E61201A0743A5F
:1005900012010F08E61201A012015690074312053E
:1005A000E108E67F0833F5F04007742D12010F8053
:1005B00005744F12010F120156E5F0DFE812013FFA
:1005C0000880B41201350204367521007590FF12BF
:1005D00003261201350204361203261201350204E5
:1005E00036E493B4100122C082C08312010FD0837D
:1005F000D082A380EC0D0A4D696E696174757265D5
:10060000205265616C74696D6520436F6E74726F02
:100610006C6C6572205254432D333730370D0A44C9
:10062000657369676E6564206279205769636869DC
:1006300074205369726963686F74650D0A2620100F
:100640000D0A6F20202072657475726E2070726FB3
:100650006D70740D0A7420202073656E64207469B7
:100660006D650D0A7A20202061646A2E2074696D00
:100670006520626173650D0A65202020656E7465D2
:10068000722063757272656E742074696D650D0AEF
:1006900064202020656E7465722063757272656EC9
:1006A0007420646174650D0A732020207374726F66
:1006B0006B652073657474696E670D0A7020202065
:1006C00070726F6772616D2074696D65720D0A7268
:1006D000202020726561642070726F6772616D0DF9
:1006E0000A63202020636C65617220492F4F0D0A38
:1006F0002F20202073656E642074696D65206F6EF5
:1007000063650D0A3F20202068656C7020636F6D63
:100710006D616E640D0A1050726F6772616D2073A7
:10072000746F7265640D0A100D0A52656164792058
:10073000746F20726563656976652070726F677289
:10074000616D104F5554505554205B312E2E385D3D
:1007500020100D0A456E7465722063757272656EA5
:10076000742074696D65203E20100D0A456E746515
:10077000722063757272656E742064617465203EC8
:0E0780002010454F4610574841543F0D0A10B7
:00000001FF
